:0400000002010032C7
:01000B0032C2
:0100130032BA
:01001B0032B2
:0100230032AA
:01002B0032A2
:0800E0007665723A20322E37DA
:0F0100007581417531007532007530007533001F
:0F010F00753400753500753600C229C22AC297B3
:0F011E00C295120170C225C2267E007B007A06B0
:0F012D00740F900000783774FFF608DAFC78370B
:0F013C007580FF74FE7F06302504D226C225FA97
:0E014B007580FFF5A0E6081FF580EA23C0E0EE
:0E0159001201B8D0E0BF00E93026D62025D331
:100167001201F6C226D2B680CAEAC0E07B80783791
:100177007580FF74FE7F06FA7580FFF5A0E6081FFD
:10018700F580EA23BF00F0DBE5D0E0FA22EAC0E021
:0F0197007B4078377580FF74FE7F06FA7580FF16
:1001A600F5A0E6081FF580EA23BF00F0DBE5D0E006
:0F01B600FA2220B00574000201DD20B1057401AA
:1001C5000201DD20B20574020201DD20B3057403CE
:0F01D5000201DD20B41A7404C0E0EF75F005A438
:0F01E400F5F0D0E025F0FCD2252024051204927E
:1001F300D22422C2241202DCB48018D22A753921F7
:0F020300753AFF753BFF753CFF753D00753E007A
:10021200753F0022B48106D22912036422B4821BE4
:10022200E5312401F531500F0532E53233333333F2
:10023200500575320F153112036422B48322C2288D
:0F024200E531C39401F5315002D228E532940022
:10025100F5325009753200302803753100120364FC
:0F02610022B4840B302702C227302903C229227E
:10027000202949202A0B7A06783774FFF608DAFC21
:0F02800022C0E0940A5027D0E0E53EF53FC0E0F1
:10028F00E53DF53EC0E01202DCF53D1202E2F53924
:0F029F00D0E01202E2F53AD0E01202E2F53B2283
:0E02AE00D0E0C22A1203A81202F21203642248
:0F02BC001202DCC0E012033AD0E01202E2F53881
:1002CB007537FFE5312401F5315002053212036415
:1002DB00229004ADEC9322B4FF0374FE229004CB66
:0F02EB00932290052B9322753100753200E53177
:0F02FA00F533E532540FF5F0E536C454F025F036
:10030900F534E536C4540FF535120456C0E094802F
:0F031900501CD0E0F53751ED1203CAC2B6E537DC
:0F03280051E2F5373170D2B631941203BF80C164
:0F033700D0E022C0E0E531F533E532540FF5F0A8
:10034600E536C454F025F0F534E536C4540FF535DA
:10035600120456B4FF05D0E071FD22D0E022E5314B
:0F036600540F51E2F539E531C4540F51E2F53A25
:0F037500E532540F51E2F53BE532C4540F51E22B
:0F038400F53CE531F533E532540FF5F0E536C4BD
:1003930054F025F0F534E536C4540FF53512045600
:1003A30051E2F5372275F00AE53EA4C0E075F0642A
:1003B300E53FA4D0F025F0253DF53622E5312401B3
:0F03C300F5315002053222135005D2900203D4B7
:0F03D200C290135005D2910203DEC29113500561
:0F03E100D2920203E8C292135005D2930203F2A4
:0F03F000C293135005D2940203FCC29422C0E0C2
:0F03FF00C2B51204907406120481120490D2B594
:0F040E00120491C2B51204907402120481E535F4
:0F041D00120481E534120481E533120481D0E02A
:10042C00120481120490D2B5120491C2B512049137
:0F043C0074051204817400120481C0E012049050
:10044B00D2B5D0E0B400E212049122C2B5120490EE
:0F045B007403120481E535120481E53412048123
:0F046A00E5331204817400120481C0E012049083
:0F047900D2B5120491D0E0227F08339295D2972A
:0F048800A29633C297DFF5222222202A0651DCEA
:0F049700947F40012251DCC0E051E2F537D0E004
:1004A60051ED71CAC2B622000000000080474D41DE
:1004B6000A810708090B820405060C830102030D55
:1004C6008454000F0E21E732A2E4A828E320A02ED0
:1004D6002C3E263878FFFFFFFFFFFFFFFFFFFFFFE1
:1004E600FFFFFFFFFFFFFFFFFFFFFFFFFFFFFFFF16
:1004F600FFFFFFFFFFFFFFFFFFFFFFFFFFFFFFFF06
:10050600FFFFFFFFFFFF60FFFFFFFFFF29FFFFFF6A
:10051600FFFF61FFFFFFFFFFFF79FFFFFFFFFFFF09
:10052600FFFFFFFFFF000102030405060708091885
:10053600191A1B1E1FFFFFFFFFFFFFFFFFFFFFFF35
:10054600FFFFFFFFFFFFFFFFFFFFFFFFFFFFFFFFB5
:10055600FFFFFFFFFFFFFFFFFFFFFFFFFFFFFFFFA5
:10056600FFFFFFFFFFFF14FFFFFFFFFF12FFFFFF6D
:10057600FFFF13FFFFFFFFFFFF17FFFFFFFFFFFF59
:05058600FFFFFFFFFF75
:00000001FF
